:100000002828A301A200FF30A207031CA307031C9A
:1000100023280330A100DF300F200328A101E83E90
:10002000A000A109FC30031C1828A00703181528FC
:10003000A0070000A10F152820181E28A01C2228A8
:100040000000222808008313831203130000080015
:10005000073099003230A4003230A500051E3A283E
:1000600083160510831205108316851083128510E0
:100070003B283B288C28A7010330270203186B2854
:10008000A601043026020318542883160510831293
:100090000514240801208316051083120510250875
:1000A0000120A60A031D4128A601043026020318D8
:1000B000682883168510831285142408012083166E
:1000C00085108312851025080120A60A031D5528D6
:1000D000A70A031D3C28A7010330270203188B2819
:1000E00083160510831205142408012083160510B9
:1000F00083120510250801208316851083128514AC
:1001000024080120831685108312851025080120FC
:10011000A70A031D6C282E288316051083120514C8
:0E01200083168510831285142E2863009528FF
:02400E00E43F8D
:00000001FF
